:0200000480007A
:100000006F00C004732F2034930F8000630AFF0336
:10001000930F90006306FF03930FB0006302FF038A
:10002000170F0080130F0FFE63040F0067000F000F
:10003000732F203463540F006F004000136E9E53E3
:10004000171F00002320CFFD6FF09FFF732540F1A5
:100050006310050073251030635805000F00F00F82
:10006000130E100073000000130E00009702000032
:10007000938282F973905230735020307350303035
:1000800073504030970200809382C2F7638C020065
:10009000739052109302B01A739022307323203061
:1000A000E39E62F873500030970200009382420191
:1000B00073901234732540F173002030B700008034
:1000C00013010000B3D12000B70E0080130E2000F2
:1000D0006398D157B700008013011000B3D12000FE
:1000E000B70E0040130E3000639CD155B70000805E
:1000F00013017000B3D12000B70E0001130E4000B1
:100100006390D155B70000801301E000B3D1200007
:10011000B70E0200130E50006394D153B700008055
:10012000938010001301F001B3D12000930E100052
:10013000130E60006396D1519300F0FF130100008D
:10014000B3D12000930EF0FF130E7000639AD14FCD
:100150009300F0FF13011000B3D12000B70E008010
:10016000938EFEFF130E8000639CD14D9300F0FF31
:1001700013017000B3D12000B70E0002938EFEFF72
:10018000130E9000639ED14B9300F0FF1301E0002B
:10019000B3D12000B70E0400938EFEFF130EA00013
:1001A0006390D14B9300F0FF1301F001B3D1200015
:1001B000930E1000130EB0006394D149B720212193
:1001C0009380101213010000B3D12000B72E21211B
:1001D000938E1E12130EC0006394D147B7202121C5
:1001E0009380101213011000B3D12000B79E90101D
:1001F000938E0E09130ED0006394D145B7202121B0
:100200009380101213017000B3D12000B74E42004A
:10021000938E2E24130EE0006394D143B720212146
:10022000938010121301E000B3D12000B78E0000BC
:10023000938E4E48130EF0006394D141B7202121D4
:10024000938010121301F001B3D12000930E00002F
:10025000130E00016396D13FB72021219380101225
:10026000130100FCB3D12000B72E2121938E1E1262
:10027000130E10016396D13DB720212193801012F7
:10028000130110FCB3D12000B79E9010938E0E097D
:10029000130E20016396D13BB720212193801012C9
:1002A000130170FCB3D12000B74E4200938E2E2470
:1002B000130E30016396D139B7202121938010129B
:1002C0001301E0FCB3D12000B78E0000938E4E489E
:1002D000130E40016396D137B7202121938010126D
:1002E0001301F0FFB3D12000930E0000130E500154
:1002F0006398D135B700008013017000B3D020009F
:10030000B70E0001130E6001639CD033B70000806C
:100310001301E00033D12000B70E0200130E70016C
:100320006310D13393007000B3D01000930E00001F
:10033000130E80016396D03113020000B7000080D5
:1003400013017000B3D120001383010013021200C7
:1003500093022000E31452FEB70E0001130E900129
:100360006310D32F13020000B70000801301E000D8
:10037000B3D1200013000000138301001302120008
:1003800093022000E31252FEB70E0200130EA001EA
:100390006318D32B13020000B70000801301F00193
:1003A000B3D12000130000001300000013830100EC
:1003B0001302120093022000E31052FE930E10006D
:1003C000130EB001631ED32713020000B700008094
:1003D00013017000B3D12000130212009302200019
:1003E000E31652FEB70E0001130EC001639AD12529
:1003F00013020000B70000801301E00013000000AA
:10040000B3D120001302120093022000E31452FE25
:10041000B70E0200130ED0016394D1231302000023
:10042000B70000801301F00113000000130000006A
:10043000B3D120001302120093022000E31252FEF7
:10044000930E1000130EE001639CD11F13020000F5
:10045000B70000801300000013017000B3D120002A
:100460001302120093022000E31452FEB70E0001A3
:10047000130EF0016396D11D13020000B700008037
:10048000130000001301E00013000000B3D12000AE
:100490001302120093022000E31252FEB70E020074
:1004A000130E0002639ED11913020000B7000080F2
:1004B00013000000130000001301F001B3D120006D
:1004C0001302120093022000E31252FE930E10005A
:1004D000130E10026396D11713020000130170006F
:1004E000B7000080B3D12000130212009302200055
:1004F000E31652FEB70E0001130E20026392D115CF
:10050000130200001301E000B70000801300000098
:10051000B3D120001302120093022000E31452FE14
:10052000B70E0200130E3002639CD11113020000BB
:100530001301F001B7000080130000001300000059
:10054000B3D120001302120093022000E31252FEE6
:10055000930E1000130E40026394D10F130200009B
:100560001301700013000000B7000080B3D1200019
:100570001302120093022000E31452FEB70E000192
:10058000130E5002639ED10B130200001301E00012
:1005900013000000B700008013000000B3D120005A
:1005A0001302120093022000E31252FEB70E020063
:1005B000130E60026396D109130200001301F001CB
:1005C0001300000013000000B7000080B3D120002A
:1005D0001302120093022000E31252FE930E100049
:1005E000130E7002639ED1059300F000335110008A
:1005F000930E0000130E80026314D10593000002D5
:1006000033D10000930E0002130E9002631AD1033F
:10061000B3500000930E0000130EA0026392D003AB
:1006200093000040371100001301018033D02000F7
:10063000930E0000130EB0026314D001631CC001BE
:100640000F00F00F63000E00131E1E00136E1E003D
:10065000730000000F00F00F130E10007300000075
:10066000731000C000000000000000000000000047
:10067000000000000000000000000000000000007A
:040680000000000076
:1010000000000000000000000000000000000000E0
:1010100000000000000000000000000000000000D0
:1010200000000000000000000000000000000000C0
:1010300000000000000000000000000000000000B0
:081040000000000000000000A8
:040000058000200057
:00000001FF
